:020000020000FC
:100000007AC007C05DC05DC05DC05DC06CC06CC023
:100010006CC04FB7662412B7412E15B710FB4EF1D6
:10002000116015BF19E3411A312C332021F4C09817
:100030001FEF1EBD43C011E0311A21F0C09A1FEF1F
:100040001EBD3CC013E6411A40F440941CE1410E31
:1000500013E2141948F4C09808C01CE1410E13E2E1
:10006000141910F4C09A01C044248894440C4EBC66
:1000700025C01E7F15BF19E312BF212C112413E1E7
:10008000121960F417E1121948F01FE1151969F00F
:1000900060F0539414E1151940F00CC0552051F054
:1000A0005A9414E1151908F005C010B7106610BF76
:1000B000C49A04C010B71F7B10BFC4984FBF1895D7
:1000C0001895189518954FB719E312BF612C12E3D4
:1000D000161910F0139405C010B71F7B10BFC498F9
:1000E00055244FBF189518951895189558B361E089
:1000F000562758BB089503E005BF00E40BBF02E09C
:1001000009BF02E003BF06E200BFA89500E001BD01
:1001100003E107BB002708BB03E008B902E207B907
:1001200003E006B90FEF0DBD00E00EBD08E601BF0C
:06013000C4987894FFCF93
:00000001FF
